:100000000C9434000C9451000C9451000C94510049
:100010000C9451000C9451000C9451000C9451001C
:100020000C9451000C9451000C9451000C94AB00B2
:100030000C9451000C9451000C9451000C945100FC
:100040000C9451000C9451000C94C2010C9451007A
:100050000C9451000C9451000C9451000C945100DC
:100060000C9451000C94510011241FBECFEFD8E026
:10007000DEBFCDBF11E0A0E0B1E0EEEFF4E002C0E2
:1000800005900D92A830B107D9F713E0A8E0B1E0D0
:1000900001C01D92A832B107E1F70E9453000C94F1
:1000A0007D020C9400000E942D020E94EA007894C8
:1000B00081E080932603C1E008E012E00F2EF5E115
:1000C000EF2EF2E0FF2EF02D0F2EF2E2CF2EF2E017
:1000D000DF2EF02D0F2EFEEFAF2EF1E0BF2EF02D14
:1000E000809126038823E1F7C09326030E9405012F
:1000F000809127038133A1F7C8010E9445028AE05D
:100100000E9425028DE00E942502809127030E9413
:1001100025028AE00E9425028DE00E942502C70187
:100120000E9445028AE00E9425028DE00E9425027D
:10013000C6010E9445028AE00E9425028DE00E94CD
:100140002502C5010E9445028AE00E9425028DE039
:100150000E942502C5CF1F920F920FB60F92112455
:100160002F933F934F935F936F937F938F939F93BF
:10017000AF93BF93EF93FF9384EF8093890084E262
:100180008093880084E50E942502809126038823BD
:1001900029F080912603815080932603FF91EF91EF
:1001A000BF91AF919F918F917F916F915F914F918F
:1001B0003F912F910F900FBE0F901F90189583E0E5
:1001C00084B90895289A089528980895299A089539
:1001D00029980895E1E8F0E080818860808380813B
:1001E0008460808380818160808384EF8093890034
:1001F00084E2809388001092850010928400EFE6DC
:10020000F0E080818260808308952F923F924F9228
:100210005F926F927F928F929F92BF92CF92DF9266
:10022000EF92FF920F931F93CF93DF93F894C090B8
:100230002403DD241C141D040CF084C0B09027039B
:10024000A0E3B2E020E030E000E010E0EE24FF2484
:10025000C0E0D0E060E070E00F2EF2E26F2EF2E03E
:100260007F2EF02D0F2EF5E14F2EF2E05F2EF02DB8
:100270000F2EF8E08F2EF2E09F2EF02D0F2EFEEFC6
:100280002F2EF1E03F2EF02D2130310541F4F40105
:10029000E00FF11F8C9180830F5F1F4F19C0A901E0
:1002A000C90102978230910540F4F201EE0DFF1D65
:1002B0008C9180830894E11CF11CCA010497823060
:1002C000910530F4F301EC0FFD1F8C918083219692
:1002D00026303105C1F4C401800F911F0197FC0144
:1002E0001082C2018E0D9F1D0197FC011082C30177
:1002F0008C0F9D1F0197FC011082FD013197B0808A
:10030000C0E0D0E009C02930310531F4F101EC0F33
:10031000FD1F8C91808321968D918C3211F42F5F7B
:100320003F4F2A30310534F0B0922703C350DE4FDF
:10033000188208C06F5F7F4F6C157D050CF4A4CF49
:10034000B09227037894DF91CF911F910F91FF9086
:10035000EF90DF90CF90BF909F908F907F906F90A5
:100360005F904F903F902F900895F894E8E0F1E06F
:100370008DEF91E01192E817F907E1F71092FC0177
:10038000789408951F920F920FB60F9211242F9315
:100390003F934F935F936F937F938F939F93AF930D
:1003A000BF93CF93EF93FF93C091C6008091FC0160
:1003B000833F50F4E8E0F1E0E80FF11DC0831182C3
:1003C0008F5F8093FC010CC00E94B5018091FC01FD
:1003D000E8E0F1E0E80FF11DC0838F5F8093FC013E
:1003E00080912503813069F088E091E060E071E060
:1003F0000E946302009729F081E0809325030E9408
:10040000B501CA3281F480912503813061F480E323
:1004100092E068E071E00E945C028091FC018093B0
:10042000240310922503FF91EF91CF91BF91AF91DB
:100430009F918F917F916F915F914F913F912F91FC
:100440000F900FBE0F901F901895E0ECF0E0908198
:1004500095FFFDCF8093C60008951092C50087E6F2
:100460008093C40088E98093C10086E08093C20035
:1004700081E40E9425028BE40E9425028AE00E940A
:1004800025028DE00E9425020895CF93DF93EC01B1
:100490008881882331F021960E9425028991882342
:1004A000D9F7DF91CF910895E0ECF0E080818823C7
:1004B000ECF78091C6000895FB01DC0101900D92DC
:1004C0000020E1F70895FB0151915523A9F0BF01E8
:1004D000DC014D9145174111E1F759F4CD0101902F
:1004E000002049F04D9140154111C9F3FB01411124
:0E04F000EFCF81E090E001970895F894FFCFE0
:0804FE0024475047474100006C
:00000001FF
